:1000000002780030B402D25202180B758C10D26BF9
:100010000216B630B502D25102189A32FFFFFFFF26
:10002000FFFFFF32FFFF020032FFFF36304455561C
:1000300020208520F0E4787FF6D8FD85F02090E838
:1000400000E4F0A374EFB583F874EFB582F3A20374
:10005000920190006D75A0C078007402F208E493DC
:10006000F2A308046023E493F2A30880ED16A81518
:100070005527F0067D07810982251C10371F561F62
:100080003622C50AF00AE1FFFFC20430961D309700
:100090001A7C14C296209713D29630970EC29720DE
:1000A0009609D297309604DCEAD204D296D2977D94
:1000B000177C920D9043C075A0807800E493F2A362
:1000C00008B8000205A0DCF4DDF27583F41280604C
:1000D00090F408787775F00312807990F409E03095
:1000E000E00690F40BE080F3D200743F1243BF901F
:1000F000E7FE1243BF4017F0A3B4030040121243BF
:10010000BF400BF0A31243BF4004F0A38002C20023
:100110001243BF74541243BF122881122FF3743557
:1001200012300C121BCB50726F6772616D206368C6
:1001300065636B73756D202D2D2D2D2000E4FBFF65
:10014000900000C374C0246CFC7443341C04FDBCD8
:1001500000011DE4932BFBE43FFFA3DCF6DDF4A3D9
:10016000A3E4932B7006A3E4932F600B122FFE12CF
:1001700022B47590FD80FE1222A9300033121BCBF1
:100180004F7665726C6179207265766973696F6EFE
:10019000202D2D2D2D20200090E7FEE02430A312ED
:1001A0001C06E02430A3121C06E0121C061222BE1C
:1001B0007583F01280607583F412806090F4187873
:1001C0008875F003128079745A12251C741CFD1274
:1001D000251C746CFC12251C9043C00DE493122561
:1001E0001CA3DCF8DDF6E493A312251CE493A31210
:1001F000251C74A13002027461FE7C007940C0E0CD
:1002000090F419E030E00690F41BE080F3D0E07D3C
:100210000512251C12024512253AF7543F500AF8E0
:10022000EEC4440F68D36001C3EC92E303FC090EF3
:10023000EE30E2DB90023DEC93F57780110307008E
:100240000B0000000F7B127A00DAFEDBFC22121B8F
:10025000CB546F74616C20706F72747320666F750D
:100260006E64202D2D2D202000AD770D7A00120B0D
:10027000051222BE743612300C1209EBE577B40475
:1002800000500302037824FD0303FCA20592F779D2
:1002900040E70965F054806003757700DCF3121BBA
:1002A000CB536C61766520636F6D6D756E696361AC
:1002B00074696F6E202D2000C3E57760061222A9B5
:1002C0000203781222B47C017940121BCB20536CBC
:1002D00061766500AD047A00120B05E76068F5F001
:1002E000121BCB2020526F6D3A2000A2F012036443
:1002F000121BCB202052616D3A2000A2F112036440
:10030000121BCB2020492F4F3A2000A2F212036487
:10031000121BCB202050676D3A2000A2F312036419
:10032000121BCB2020547970653A200020F70B1265
:100330001BCB4D554C544900801D121BCB50432FF5
:100340004D4143008011121BCB20204E6F2072655F
:1003500073706F6E7365001222BE090CBC040280BC
:10036000170202CA4009121BCB424144200022124C
:0F0370001BCB474F4F440022E577700812300532
:10037F007590FE80FE90E865F0743712300C12090C
:10038F00EB30030812333A500302042675A0E979C3
:10039F00009064007D017C507F007B00E493F3129A
:1003AF000436A309B9000205A0DCF1DDEF75A0EA60
:1003BF0079009065007C00E493F579E493F31204DF
:1003CF0036A309DCF6121BCB436F6E666967206399
:1003DF006865636B73756D20202D2D2D2D2000907A
:1003EF0067FEE4932B7027A3E4932F702190E9000D
:1003FF00E0B4011A90E901E0B4231390E902E0B4EC
:10040F00010C90E903E0B404051222A980301222F6
:10041F00B47590FF123019120824400612302302CF
:10042F00039B12302A80ED2BFBE43FFF22012301B7
:10043F00040005100F2B00101A000021000090E996
:10044F0004E0A2E09238A2E1922490E905E090E85E
:10045F006EF0A3F090E906E090E86CF0A3F090E95D
:10046F0007E0F57790E908E090E863F090E909E09C
:10047F0090E86AF0A3F090E90AE090E868F0A3F042
:10048F0090E90BE0F55F90E90CE0F57690E90DE06F
:10049F00F57890E866F090E90EE090ED00F030020C
:1004AF000990E865E0F57F0228A81280115389F0C2
:1004BF00438901D28CD2A9D2AF7551607550607546
:1004CF005A4075594012067D306E1F74201285FAFE
:1004DF00121BCB5043206B6579626F61726420648D
:1004EF00657465637465640D0A001207D112078184
:1004FF00303908121D20755F12804030251F121BE6
:10050F00B90D0A00121BCB50532F32206D6F75732C
:10051F00652064657465637465640D0A00206E035D
:10052F001206E5306E1220390FA201C0D0C201129F
:10053F0021D3D0D09201C25C1280FD1209F4D2688F
:10054F00D26E757B00757C0090E8577406F090E8CA
:10055F00507400F0A3F01230347405304D0274045F
:10056F00A201C0D0C201D26A122488D268120A70C6
:10057F00D0D0920120010302063E121BCB0D0A5070
:10058F007265737320009005E3122F999005F9128D
:10059F002F992003581205AC1205BA8056121BB9B9
:1005AF00656E746572206B65790022121BE7656EAC
:1005BF00746572206F6E206B6579706164002230F4
:1005CF0098FDC298E5992212333A400122B40702EE
:1005DF00D322C322C048697420656E74657220747B
:1005EF006F2070726F63656564009320001205AC15
:1005FF001205BA121BCB20746F20636F6E74696E75
:10060F0075650D0A00E41243BF43900320031212D5
:10061F0005D640093098F81205CEB40DF2D2D1802C
:10062F000E1205D640093098F81205CEB40DF243DC
:10063F007DC3C203E41243BF1243BFA25D924AC2FD
:10064F005D1218FAA24A925D1285C8B3921B122F3F
:10065F0085200015121BCB0D0A5374617274696EDD
:10066F0067206D61696E0D0A00C201020B2DC2A8D1
:10067F00D21F90E88574FAF0E55F540FB40548C2B5
:10068F00AA1207ECC2B2120245D2B3780F128669D2
:10069F007C32120245DCFBC2F090F401E030E02620
:1006AF0054E07900600279FF5382F8438203E0B986
:1006BF0000E720F00AB4FEE112902ED2F080DA901B
:1006CF00ED00F01285DC22B40408C2AA124344D212
:1006DF00B3221207B622206E7575B0FF7A0A79140D
:0E06EF00E5B0543CF8E5B0543C687009D9F70A
:1006FD00E854246424600CDAE9121BCB0D0A504334
:10070D000080537850D8FE7904B2B27850D8FEA24A
:10071D00B413A2B513D9F2D2B2B4CC14755F44128E
:10072D00067D120781121BCB4170706C650080260F
:10073D00B488028003B4DD18755F5512067D12076B
:10074D0081121BB90D0A00121BCB53756E0080066A
:10075D00121BCB504300121BCB206B6579626F616E
:10076D007264206361626C65206465746563746591
:10077D0064200022C225C24DE55FB455061207EC78
:10078D00C2AA22B44403C2AA2220391954F0B4508B
:10079D000122B4200D1207EC1209EB121C398559F8
:1007AD005A22B4100312221322752508D288D2A81A
:1007BD00C289D2B2122196400AD26EB4EF05D23957
:1007CD0075516022752608D2BAD28AC28BD2AAD2AE
:1007DD00B31209EB1221B34005D2251221B322E544
:1007ED005FC4540775F000B40304D2F08005B4055E
:1007FD0002D2F07866C2F190F40012807990F41074
:10080D0012807912081422D2EE12081BC2EE790062
:10081D007A40D9FEDAFC22121BCB52656C6F6164F3
:10082D00696E67204E5672616D20746F206661632C
:10083D00746F72792064656661756C740D0A0012AF
:10084D00304C1209827B007F0075A0EB790090047B
:10085D003C7C00E4BC5000502EBC4000400890434E
:10086D00BFEC540F801BBC3000400474108018BCCA
:10087D00200040047401800FBC10004004740280FD
:10088D000693BC0702E577F3120436A3090CBC00EE
:10089D00C290640012091250012290EB007C00748A
:1008AD0012F0120436A3DCF7906500120912500104
:1008BD002290EB007C40E4F0A3DCFB7E0890660008
:1008CD00BE010E75A0EB793EC3E49BF309C3E49F13
:1008DD00F375A0EB79001216A85002D322DEE17B4E
:1008ED00017E40906800C082C083C00612093AD0D4
:1008FD0006D083D08275A0EB79001216A85002D3D2
:10090D0022DEE3C3227C0075A0EB7900EC2582F595
:10091D0082EC29F9C004C082C0831216A8D083D0FE
:10092D0082D0044007EC2440FC70DCC32278049094
:10093D00EB00D2217C00EC242B83F0BC081CBB0007
:10094D00067D007A0180048B057A00C000C0061276
:10095D0022C5D006D0007C0B8002A30CBC10D70B97
:10096D00D8D2C22122436F6D70757465722020201C
:10097D00202020202090099A75A0EF7980E493F330
:10098D00A3097409B583F674EBB582F122C083C057
:10099D008290555574AAF0902AAA7455F090555529
:1009AD0074A0F0D082D083C083C082C0017C40E3AC
:1009BD00F0DC02800409A380F6C3F8E493684004D8
:1009CD0030E7F8D320E7F4D001D082D0837C40E427
:1009DD0093F8E3A309B50004DCF5C322D322780014
:1009ED007900D9FED8FC2274E612251C7C01EC128C
:1009FD00251C90ED00E0A312251CDCF990E9147E76
:100A0D0004120A6190E9247E14120A6190EA047EB0
:100A1D0024E578603790E930E0FA8578F0A4240475
:100A2D00C39578F5827583EA7C0C7905EE12251C49
:100A3D000EE578B501005005E07A018002741212BE
:100A4D00251CE5822AF58209DCE28003120A61E4A5
:100A5D0012251C227C0CEE12251C0EE0A312251C67
:0E0A6D00DCF422E578B4010040567C00BC04A5
:100A7B0000C00450168C74741612814E120ACE7478
:100A8B0005304D02740412814E802F74011224889C
:100A9B00ECC412248874EF12248874161224881262
:100AAB000ACE7405304D027404C0E074EF12248832
:100ABB00D0E01224887416122488E578D0040CB583
:100ACB0004AC22C0E0C082758205E4D5E0FDD5827E
:100ADB00F9D082D0E02275F010A42400F582E5F065
:100AEB003468F58322120AE15382C075A0EB7900BA
:100AFB007C40E493F3A309DCF922300124D221904A
:100B0B00E810C004C0011222C5C2217C0390E8107A
:100B1B00E01285FA3000031243BFA3DCF3D001D0FF
:100B2B000422306B0A90E886E0D2E6F01216C9E593
:100B3B005C7013304C051221D3C24C306D08120778
:100B4B0081128FC4C26D12307990E866E0F578207F
:100B5B003937E55F54F0C4B4041ED55B2C755B10BC
:100B6B00E579B45503755B64E55C70031241F3E5FD
:100B7B005370161241978011B40508121C13121CE6
:100B8B00398006B40203121C39205E0C20700C2035
:100B9B007109206F06020BEB020E1BE55C60152042
:100BAB007209D27290E83FE4F0803590E83FE0B4F0
:100BBB000200402C7D03C27230251574F5122125DD
:100BCB002067071221B340028006DDEAC225C24D21
:100BDB00D27F75260885595A755C00D25F1218FAB8
:100BEB0030195912253A5054120BF8804F12900BB2
:100BFB00F830E737B485005003D2682230E617533C
:100C0B0000071210375407B40400502FE054F0487B
:100C1B00F0F579D25D2230E505A2E0921B2230E49B
:100C2B001AD25C128FEEE8540FF0227583E8E5754B
:100C3B00C4540F4440F582E8F0D275221286F54079
:100C4B0003020E98307A03020CFE30272B90E850EB
:100C5B00E0F8A3E0C868601E75A0ECE2F5567009D9
:100C6B0008B8C0027800E2F557D27A08B8C002780B
:100C7B0000E8F0020CFEC227207678E550B5510251
:100C8B008071E55FB444028022B45502801DA851E7
:100C9B00E6B4F706D211D2148007B4F80EC211D203
:100CAB0014E55104546FF551020E1B121C593001FF
:100CBB000F307A0CE5561290517005E55712905192
:100CCB00102302802EE550B55109303BF8D2B2C249
:100CDB003B80F212111712901502232CE550B551DF
:100CEB0009303BF8D2B2C23B80F212111712901AA4
:100CFB0002244F307B131243BF207B0AD25D30544A
:100D0B0005121555C254020E1B20270E207C030220
:100D1B000D281230854003020E1B020D6C20394149
:100D2B00307A3EE556B44A05432C0F8034B4CA1CC6
:100D3B0020532EE52C540FB40F1E532CF0E55F54AB
:100D4B000FB40504D2538019D2768015B42D093017
:100D5B005306D276C2538009E4F57A522CC25EC296
:100D6B0053301940307A6B306868E5561290067034
:100D7B0001F4FE12251C1224DD5026B48123C26817
:100D8B00BEFF0DE557B41900400FA21892E680097B
:100D9B00E55654FCB42808E55712900112251CC2E5
:100DAB007A020E0FE5537050307A27C27AE556540B
:100DBB00FCB428258556F090E82075552030F105B8
:100DCB0074E0120DDF30F00574F0120DDFE55712F1
:100DDB000DDF803CF0A3055322301810E556700C44
:0F0DEB00E557B41900400512814E8018128C6D27
:100DFA00E5536011755520C27A75A0E8A855E2F846
:100E0A001281DF400C307609E5537005C276021074
:100E1A007F307302800AE559B55A028003121F6EA9
:100E2A00E55C700F307367128E23E55C6060755E57
:100E3A0028C27375A0E8A95EE3F830194E30684EEF
:100E4A0090F41A7415F07582187407F090E828E087
:100E5A0012901012251C1224DD5017B48314C26894
:100E6A007C0390E829E0A312901012251CDCF67589
:100E7A005C0090F419E030E3FC30E2F990F41A7463
:100E8A0015F07582187403F0020E9812823C1281D2
:100E9A005F304F07302622C226C24F105A401059DF
:100EAA002A10584F203D54105D75103C0F105C0FEE
:100EBA00105B12105F1210750902102C020F3F020C
:100ECA000F9E020FEC020F60020F6A128FEE540798
:100EDA00303905A21BB392E7120F8302102C1210AD
:100EEA004B203905B40302D23CA23992E7120F8390
:100EFA0002102CE576120F8302102C90E877E0049A
:100F0A00F0A2E01403C2E790104293600840028006
:100F1A000874FC8004C23D74F4120F8302102C2062
:100F2A003909E55F5407B40400500774F0120F83BF
:100F3A00D25A02102C207B10E579540FB404028097
:100F4A0003B4050474F88009D23D90E877E4F0749C
:100F5A00FAF18302102C74F1120F83D25802102C6A
:100F6A0030251385595A12228B74F41221252067D1
:100F7A00051221B3C27F02102CC2267905C0E012E5
:100F8A0020CED0E0306605303902D9F1D24F90E850
:100F9A0087E4F022128FEEF8E55F540FB40407E8F5
:100FAA0012439102102CB40525C000780E128669EE
:100FBA00D000E8A2E092F2A2E192F0A2E292F3A2B9
:100FCA00E392F153F00FA8F012866902102C7D0A01
:100FDA0074ED120F83303905306602DDF3D25902FF
:100FEA00102C7583E8E575C4540F4440F582E0F887
:100FFA00E55F540FF9E579540FB404028024B4056F
:10100A0012B80E03020F9E203912B90515E812868E
:10101A0069800FB8ED03020F9EB9ED06E8120F833F
:10102A008000C275205E03020B2D02108F7583EAC1
:10103A00E5764400F582E0223919111259147658DE
:10104A0000E57954077802B4030040027803E55FAB
:10105A0054FC4500F55F30391AE579D2F054F06056
:10106A0002C2F0E57954077803B404005005A2F0EF
:10107A0092E422E82290E873E551F0757E00D25E90
:10108A0090E884E4F090E884E0B420030211BAC343
:10109A00E55024109551540FF8E55F540FB4041B22
:1010AA00B802004059121117FE12111730E74CCE40
:1010BA0020E74853067F6E7042803BB405234021E7
:1010CA00B803004039121117FE12111730E72CCE5F
:1010DA0020E72853067F6E7022121117B47F1C80F6
:1010EA0015B803004018121117FE121117B4F00BAD
:1010FA001211176E7005121124704C0211C3E860A8
:10110A0009A851860612112460F1020B2DA851E696
:10111A001290290853006F885122EE121C5C307A13
:10112A001DC27A9012177C008002A30CE493601609
:10113A00B556F790123DEC93B43105200008E4222D
:10114A0050042000F91422BC0A005036E57E75F0DE
:10115A000AA42C500205F0F57E85F07FE52C540F89
:0E116A00701D057AE57AB4020AE577B46300D9
:10117800500F0211D650FBE577B409005003021155
:10118800D602108ABC1300500874F72C422C0210A7
:101198008A901262EC24F6230493C0E0EC24F62330
:1011A80093C0E022C378007908102605D8FBD9F946
:1011B800D322E52C540F70030211D690E873E0F5A2
:1011C80051755800E4F57A522CC25E020E1B1211BA
:1011D800F44016F57EE577B57E00400D857E76C233
:1011E80038C270D26FC25DC25C020D63857FF0E5C4
:1011F800F0B40200500CE57E20F005600514C3220F
:1012080060FBD3224410F0A3F0A3EEF0A3F0223049
:101218003132333435363738397674706D617775D5
:10122800437973786B6F473B3A726E69642E0C6230
:101238000F465E5D00323232323232323232323270
:101248003030323030303231323232323232323281
:10125800323231313232323232321298129D12AA7F
:10126800130312B912D612EA143A1552142214278B
:10127800154C150F1459142C1436146814D614C3AD
:1012880014A6149A148514AC14B115D6142C14365B
:1012980090E868800390E86CE57FAE7E12120C023D
:1012A8000D631211F44051604FF5771218FA020DD0
:1012B80063E57F7043E57EB48000503CC082C08304
:1012C80090E863F0D083D082122200020D63E57F9C
:1012D8007026E57EB40200401F90E930F0D26F021C
:1012E8000D63E57F7012E57EB41100500BF5789020
:1012F800E866F0D26F020D630211C3E57F7040AA61
:101308007EE57E603AB40B004069B414004030B406
:101318001600402EB41E004026B42100403AB428DE
:1013280000401CB428030213EAB432004011B4325E
:10133800030213EAB43C004006B43C030213EA0279
:101348000D63E55F5407B40400500AE57EA2E0E5AA
:101358005F92E3F55F020D63E55F5407B404005044
:101368000CF9E57E24EB834501F55FD26D020D6330
:10137800102050121037D26DA97953010FB904000B
:101388004005BA06005058BA04047444803EBA05B1
:101398000474558037BA0B0474668030BA0C047430
:1013A800778029BA04004013540FCA24FBB40404FC
:1013B80074058016B405137400800FC4540FA879FF
:1013C800530007B8040040027401C44AF579D25D9D
:1013D800121037E579F0FBD24AE582FE122808029E
:1013E8000D63B428047444800CB432047455800529
:1013F800B43CEC7412FB90EA00AC770CEBF0E5829D
:10140800FEC082C083C004C0031227F0D003D004FA
:10141800D083D082A3DCE5020D63D238020D63C20B
:1014280038020D63D270C238C25DC25C8020D271AE
:1014380080F4C201E57E6016D201B4010853877FAB
:10144800758DFD8009B40206438780758DFF020DF6
:1014580063E52C540F60062409FC0211990211D689
:1014680020000312287B121B6BC238E55FB44402CC
:1014780080DCB4550280D7D24CD26D80D130000CBC
:10148800D27CD27BD25D1243BF020D63123180023F
:101498000D63D27BD25DC27C1243BF020D6312433F
:1014A800BF020D63B224020D63E579B4550A7400D6
:1014B800121F56741E121F56020D637E009028A23A
:1014C800EE936007FA121F360E80F2020D631214B3
:1014D800DC020D63E57954E0701120180F20192102
:0E14E800755C01755E2890E828E4F022E5743A
:1014F60012851B74EF128544E57412851B74311234
:10150600854422743112248822121515020D63E5D2
:101516007954E07015201813201925755C02755E44
:101526002890E82874AAF0A3E4F022E57412851B3B
:1015360074EF128544E57412851B743212854422B9
:101546007432122488221215550214560214567A41
:10155600151215671215D950002290E949E0443852
:10156600FAE578606A7B00EB12851BC023C219740A
:10157600EF128544EB12851BEA12855DD0230BBB67
:1015860004028006E578B503DE22E57824FC603F98
:10159600FB757540D219D2187401122488E57512AC
:1015A6002488D223EA122488E5752410F575120AD8
:1015B600CEDBE5741612248812197F120ACE120A9F
:1015C600CE120ACE120ACE120ACE120ACED26F223C
:1015D600020D6390E904E0A23820000292E0A22402
:1015E60092E1F090E86EE090E905F090E86CE0900A
:1015F600E906F0E57790E907F090E863E090E908FE
:10160600F090E86AE090E909F090E868E090E90A6D
:10161600F0E55FB444028003B4550474128002C23C
:10162600E090E90BF0E57890E90DF090ED00E090A0
:10163600E90EF01209827B007F007C5090E900E4FD
:1016460093120436A3DCF875A0EB790090EA007CCF
:1016560000E493F3120436A309DCF690640075A047
:10166600E979001216A850012290644075A0E97924
:10167600401216A85001229065001209125001224C
:1016860090EB007C40E4F0A3DCFB90EB3EC3E49BD4
:10169600F0A3C3E49FF09067C075A0EB7900121623
:1016A600A822128B8512EF8092F0128B5AA2F0229A
:1016B600202B06107E03752508203306107D037542
:1016C600260832C26B303B15C3E5502410955154A1
:1016D6000FB409005007752508D2B2C23B303A193B
:1016E600C3E5592410955A540FB40900500B7526BA
:1016F60008D2B3C23AD249804090E876104938E51C
:101706007454039085C49390E87645C0B4FF28E0EE
:1017160004F0B40F00501B5407B4001D755C00E5BF
:101726005AB559028011F8E6B4AA0E0853004FE6DE
:10173600700785595AD26DE4F01243BF304F1790A7
:10174600E887E004F0B4030EC24FC259C25AC25829
:10175600C25CC25DC25B2039323079173077101215
:101766001A4374311243BF1243BFC277122F85C288
:1017760079801290E8691217E25010121A19D2777E
:101786001243BF800690E8681217DA90E884E004F6
:10179600F090E83FE004F012860520111F201A1C85
:1017A600207B1930381690E86D1217E2500ED215CC
:1017B600D270C25DC25C90E86C1217DA303F1190AD
:1017C600E867E004F0B402004006121A76123255B9
:1017D60012326222E0A3F0A3E0A3F022E02410F08C
:1017E600501FF84410F0A3A3E0B80002601314F0F1
:1017F600B4FF09E81415821582F0C3227003E8606D
:1018060002C322D322202F1E302B0A105206D27971
:10181600D27E152532C55203D2E7105202C2E7C561
:10182600521525C22B32102857752508105216D28C
:1018360074C2B2C001C55264AA6006C5527930802E
:101846003864AA80173013E7C2B2C001C55264FAE1
:101856007008D226C5527930801F64FAC552A95045
:0E186600A7520953016F8950C904546F655190
:101874007006D23BC9D00132C97926D9FED2B2D082
:101884000132C552D21310520520D007800330D044
:1018940002C213C5523220372030330C105108D203
:1018A40079D27DD249152632C55B03D2E7105102A5
:1018B400C2E7C55B1526C2333210302675260810E0
:1018C400510132306C2FC001A959A75B0953014F54
:1018D4008959C904544F655A7004C2B3D23AC9D065
:1018E4000132C55BD26C10510520D007800330D083
:1018F40002C26CC55B32205E27205924205A212065
:10190400581E203D1B205C18205D15203C12205BD6
:101914000F10700D107118C26FE577B57600501B6B
:10192400220576E577B576005011757600800C15A2
:1019340076E5760470058577768000C20774AA423E
:10194400C0D21F128B211233CD2039031243BF2082
:101954004E03121A7612197F304E0D121BB92066EF
:10196400702A00C218C21922121AFD121AB41233B4
:10197400D410150122301402D25B22A976121996D2
:10198400F575A2F69219A2F79218A2F5924E128753
:101994003D22203904E5787006E9C454F0802EE530
:1019A40078B40F03E980268578F090E930E0A41438
:1019B400B50100500BC304F5F0E995F0257880DA01
:1019C40090E930E0F5F0E984540FC445F0F875F07F
:1019D4000020390BE854F0C4B578005002D2F7E87F
:1019E40054C06002D2F6C0F090E930E08578F0A4EB
:1019F400C0E0E5F06006D0E0D0F0E82290E865E0D1
:101A0400D0F025F0C39578B501005005D0F0D2F59B
:101A140022D0F0E82220180520191C801FE575C487
:101A2400540312851B74EF128544E575C4540312E4
:101A3400851B74021285447402122488C2EC22208D
:101A440019052018028028301905740C12248830D6
:101A5400181FE575C4540312851B74EF128544E501
:101A640075C4540312851B740C128544201902D2C8
:101A7400EC22C23F20191F301833E575C4540312F9
:101A8400851B74EF128544E575C4540312851B74D9
:101A940016128544801730180F74EF1224887416B8
:101AA40012248874021224887416122488C2EC2228
:101AB4002018403019337409D26A1224881224EB96
:101AC4005025D268F854706020C4B40600501AE857
:101AD400A2E7921B128FEEE8540FF0E8C45407F803
:101AE40012103754F048F08003121037F579D25DA4
:101AF400D25C22121037F5792220182F20190EE516
:101B040075C45403F57444FCF590D2EC22120ACE49
:101B1400120ACE120ACE120ACE7401122488E57576
:101B240054F0122488740C12248822201924121BC5
:101B340003E57412851B74EF128544E57412851B4A
:101B44007401128544E57412851BE575540F1285E2
:101B54004422121B1174EF1224887401122488E5A4
:101B640075540F1224882220181020193A9093EBF0
:101B7400E574540393457DF57D22301903121BABA4
:101B8400E574540312851B74EF128544E574540301
:101B940012851B7430128544E574540312851BE5C9
:101BA40075540F128544227430122488E575C45488
:101BB4000F12248822D083D082E4931285FAA3E4FE
:101BC40093B400F7740173D083D082C082C083E4DD
:101BD400931285FAA3E49370F8200007D0E0D0E0D4
:0E1BE400740173D083D082E493B40A02800DA2
:101BF20030010A300007C0011243BFD001A3E493B1
:101C020070E904733001091285FA3000031243BFF0
:101C12002290F401E030E01E54E07900600279FF86
:101C22005382F8438203E0B900E7A950F705505305
:101C3200506FD27980DB2290F411E030E0185382A9
:101C4200F8438203E0A959F7055953594F12906A94
:101C5200D249D27980E122121117F8FCAE5F530605
:101C62000FBE041B207B0BE5795407B4040040022D
:101C7200801CE820E7616439605D205E608021BEDF
:101C82000578207B10E5795407B40400400790E8FA
:101C920086E4F08048E820E73E647F603A205E3DBB
:101CA20090E886E020E7077400D2E7F0802454072A
:101CB200B40702800EE550B55102802590E8867483
:101CC20000F022E550B5510F90E886E030E61CC2E4
:101CD200E6F0121D0C800690E8867400F08C0080FD
:101CE2006C90E886E030E603121CF1121D0C229083
:101CF200E886E05487045487F022E5586003021E08
:101D020027B8AA10D26E1221D322E55114540F44DF
:101D120060F55122B8DF004034B8EF16D223D23931
:101D220074301243BF757800C23875770FD26ED205
:101D32002522B8F00475580122B8E0047558022231
:101D4200B8E1047558042275F000021DF7E55F54EE
:101D52000FB4040690265D021DE9B4052BE5795403
:101D620003B4031F90ED00E0B421028016B42202F6
:101D72008011E8A2E792F0C2E7B458077420A2F0FB
:101D8200021E1D9026DD805FC392F0E55F54039032
:101D9200254A7885B403059025CF788EECB50000EE
:101DA200505393A87920393BB844028003B8553385
:101DB200A85F53000FB80A00500CB44C02741BB455
:101DC2004B21741E801D30241AB44C04744E8013AF
:101DD200B44D04744F800CB44E04744C8005B44F5F
:101DE20002744DA2F08006E8A2E7C2E79364FF7096
:101DF2001C92F0C2F1E55F6579540370277428A242
:101E0200F092E0A2F192E1F5568C57801264FF3015
:101E1200E70975560092E7F557800492E7F556D226
:101E22007A75580022E558B401028012B40204C245
:101E3200F0800FB40305D2F0021E4C021F0CD30235
:101E42001D8BE8B4F00475580322901E87E4A39317
:101E5200A36015B500F7E49330F0022402F557753C
:101E62005600D27A75580022901E8DD2F1787FECFE
:101E7200B50000508093F5567003021DF730F00351
:101E8200435680021E211201590200000000000088
:101E92000000000000000000000000004D00004BA8
:101EA200000000000000000000004E0000000000E2
:101EB20000004F000000000000001D0000000000B4
:101EC2000000000000000000000000000000000010
:101ED20000000000005B00000000000000000000A5
:101EE20000000000005F0000000000000000000091
:101EF2000000000053005852000000505157005992
:101F0200560000000055000D547E901F2AE558939C
:101F1200B500150558E5589370117A0F121F3674E3
:101F22002D121F568002D27A755800221477E1F0E2
:101F320014F0770090E850E0F875A0ECEA7C02B467
:101F42002D027C01F208B8C0027800D2E7DCF5E885
:101F5200F0D22722C0E090E850E0F875A0ECD0E083
:0E1F6200F208B8C0027800E8F0D22722E55954
:101F70002410955A540FF8E55FC4540FB4040AB8FE
:101F800002004039121FBE8032400CB80500402DBF
:101F9000121FF740288024B4011930390280033021
:101FA0004D07B8040040168005B80300400F128F9B
:101FB000058008B803004005122060D27322A85A99
:101FC000E60853004F885A75F008A2E7B392F0A2D2
:101FD000E692E7F404A2E792F590E82FF0A85AE61B
:101FE0000853004F885AA2E692E792F490E82EF048
:101FF00090E82DE5F0F02275F008A85AE630E74E9B
:10200000F4A2E292F0A2E192F2A2E092F10853006F
:102010004FE6FE080853004F2690E82EF0EE66309B
:10202000E701B392F41853000F430040E6FE08089E
:1020300053004F2690E82FF0EE6630E701B392F59B
:102040000853004F885A90E82DE5F0F0C32208535A
:10205000004FC3E559986004E630E7F2885AD3226E
:1020600075F000A85AE630E6530853004FA2E592F7
:10207000F0A2E492F1A2E192F4A2E392F5A2E0923E
:10208000F2A2E292F3E60853004FA2F292E6C39264
:10209000F2A2F492E790E82EF0E60853004F885A37
:1020A000A2F392E643F008A2F592E7F404A2E792C5
:1020B000F590E82FF090E82DE5F0F0220853004F5E
:1020C000C3E559986004E630E6F2885AD3221290AC
:1020D0002E203B0B128B85B4FF088550518003D313
:1020E000803D7F3CDFFEC266C2B4D2B2A2D0B37CD8
:1020F000097E0A7F0030B210DFFBDEF9D2B4D2666F
:1021000080DD12216A2066171392B4122174DCF26A
:1021100012216AD2B412217412216A122174C3D21C
:10212000B4128B5A22129042128B85303A0AC23A6C
:10213000855A5980F3D3802C7F3CDFFEC267C2B53D
:10214000D2B3A2D0B37C0912217E2067171392B5B7
:1021500012218CDCF212217ED2B512218C12217E4A
:1021600012218CC3D2B5128B5A227FFF30B204DF0A
:10217000FBD266227FFF20B204DFFBD266227FFF04
:10218000780830B306DFFBD8F9D267227FFF20B38F
:1021900004DFFBD2672278007908E550B55106D8F4
:1021A000F9D9F7D322A851E61290290853006F8875
:1021B00051C322E4F8FE7902E559B55A08D8F9DE90
:1021C000F7D9F5D322A85AE612903D0853004F885C
:1021D0005AC322E55F5407B4040040012274FF1281
:1021E00020CE306601221211AC40FA7A017C001236
:1021F00021965004DCF9DAF7122200D25CD25D227B
:1022000074F31220CE1211AC90E863E01220CE12CB
:1022100011AC22C225C24D85595A74FF12212530B6
:102220006701221221B340627C031221B364AA60C9
:1022300002DCF71221B3902250E493601774F3127A
:1022400021251221B3E493A31221251221B380E9A1
:10225000C864500074F21221251221B31221B3C2B6
:102260004D6002D24D74E81221251221B37403127D
:1022700021251221B374E61221251221B312228BDB
:1022800074F41221251221B3D2252274F3122125D0
:102290002067151221B37428A8795300F0B85002B2
:1022A00074141221251221B322121BCB474F4F4425
:1022B0000D0A0022121BCB4241440D0A0022121BC0
:1022C000CB0D0A002275A0E87959E4F319F37C10CC
:1022D000C3ED33FDEA33FA75F002A801430001E2D1
:0E22E00035E0D4F218D5F0F7DCE675F003A86F
:1022EE0001D375A0E8E230F003088001C4540F500A
:1022FE000D700A20F20330F10574208003C34430C0
:10230E00302104F0A3800E305608101E08122F9EA6
:10231E0080031285FAD5F0CA302102E4F02230177C
:10232E0051C217547FF8300507540FB40400503FC4
:10233E0090E85CE0540FF94400F5827583EAE8F00A
:10234E00E9B576158879E85407B4030040047403A0
:10235E0080027402535FF8425FB90400400D74406E
:10236E0049122488E0122488020E1BE81280CA0249
:10237E000E1B30E60990E85CF0D217020E1BB41665
:10238E0010D23F90E867E4F0C259C25CC24F020E11
:10239E001BB4010B303F03121A76D21D020CE7B4A8
:1023AE000C08121A43C21D020E1BB40208121A198F
:1023BE00C21D020E1BB40410D24D7404D26A122434
:1023CE0088D268C21D020E1BB40510C24D7405D210
:1023DE006A122488D268C21D020E1BB40015740541
:1023EE00304D027404D26A122488D268C21DD25DA6
:1023FE00020E1BB4150302154CB431061214DC0286
:10240E000E1BB43206121515020E1BB43007D2483D
:10241E00C21D020CE7B4080874901220CE020E1BE7
:10242E00A2E792F0C2E7B419004013B43000500E88
:10243E00A2F092E7F557755600D27A020E1B020EE5
:10244E001B301D10540FF576C271C270C21D1218CA
:10245E00FA020E1B304811C248D26DB40400500B64
:10246E009093EB93457DF57D020E1BC0E074301208
:10247E002488D0E0122488020E1B200209F82023A3
:10248E0006B4EF03D22322306403FF8016B4010298
:10249E00800CB430028007F85300F0B84004D264C8
:1024AE00FE22FE2068051224DD50FBE412251CEEF0
:1024BE00A22392E712901F12251C306407EF129090
:1024CE002412251C106A031224DDC223C2642212B8
:1024DE0024F7500830E7F8B4850050F3221224F7A1
:1024EE0050FAF8547060F6E822C000C00178007906
:1024FE002812253A4009D8F9D9F774041285FAD072
:10250E0001D0005008C0E0120BF8D0E0D322C0E09A
:10251E0075A0F47819E230E2FCD0E0781BF2227557
:10252E00A0F47819E230E0FC781BE22290F419E076
:10253E0020E003C3E42290F41BE0D322FF09FF0541
:10254E000301020CFF0A080604462FFFFF4C48FF4A
:10255E004A7131FFFFFF7A73617732FFFF63786450
:10256E00653433FFFF447666747235FFFF6E626822
:10257E00677936FFFFFF6D6A753738FFFF416B696C
:10258E006F3039FFFF42436C3F703AFFFFFF40FF51
:10259E003C3BFFFF7C49473DFF3EFFFFFF1CFFFF1B
:1025AE00FFFF45FFFF11FF1417FFFFFF106012150D
:1025BE0016182E7B0B5E135D5C190EFFFFFFFF07D7
:1025CE007DFFFFFFFFFFFFFF012EFFFFFFFF462FE7
:1025DE0002FF4A481C7C713103FF4C7A73617732DB
:1025EE0004FF63786465343305FF44766674723590
:1025FE0006FF6E626867793607FF4D6D6A7537386C
:10260E0008FF416B696F303909FF42436C3F703AE6
:10261E000AFFFF40203C3B0B0D4B49473D3EFF0C54
:10262E000E57580F5651534550FF11591417555206
:10263E00541060121516187B5BFF5F13FF5E195C5A
:10264E00FF1B1E2DFF5DFFFFFFFFFFFF4E4F1D61A6
:0E265E0073646668677A7863761C62717765CC
:10266C007279743132333436353B39373A38303D40
:10267C006F753C6970476C6A406B3F3E41436E6DB1
:10268C004246442F45FF2E4A4F481A4C585957562C
:10269C00FFFF60FF5CFF5EFF7BFFFFFF5B5FFF5D8B
:1026AC00FFFF991011121314151617FF1819FFFFBD
:1026BC00FF050607030809FF0BFF0DFF0EFF0AFFBE
:1026CC000CFF0F505254510453025501494D4BFF0E
:1026DC001FFF9E9C9F9D01020A030B040C054D06D7
:1026EC00A90708094C560F0D0E58A0A157592E31A9
:1026FC003233343536373839303A3B2F45509B5BC3
:10270C005C1FA260A3524671776572747975696F0C
:10271C00703C3D514B1718195DA4A553FF4A6173CA
:10272C00646667686A6B6C3F403E475F1415161011
:10273C00A654A77B487A786376626E6D4142434912
:10274C00AE111213AAABAC9A7C4E444F551C5EFFD3
:10275C002D44B1C0B3B4B5B740B9B0B8BB413A42DF
:10276C004330313233343536373839BF3FC13BC251
:10277C00C3B2E1E2E3E4E5E6E7E8E9EAEBECEDEE2F
:10278C00EFF0F1F2F3F4F5F6F7F8F9FA3C3E3DB65A
:10279C00BA2F6162636465666768696A6B6C6D6E9B
:1027AC006F707172737475767778797ABCBEBDAFC1
:1027BC001B60303132333435363738392D3D5B5D63
:1027CC005C3B272C2E2F2008090D1B7E2921402332
:1027DC0024255E262A285F2B7B7D7C3A223C3E3FBB
:1027EC002008090DB576048B79D25D7583EA440017
:1027FC00F582E0B503028004D254EBF0EEF9121925
:10280C0096F920F71F20F60DE9C45403F9EB12805A
:10281C00CAD26D8041E9C4540F4440122488EB1293
:10282C0024888032E9C45403F8E9540F4440F94336
:10283C00038030F60F74EF122488E9122488EB120F
:10284C002488801274EF122869E912286974EF1237
:10285C002869EB122869204A0312408022C0E0E864
:10286C0012851BD0E0C023C219128544D02322123A
:10287C001BCB0D0A00121BCB50726F6772616D205F
:10288C007265766973696F6E202D2D2D2D2055364E
:10289C0030440D0A0022733630642D0090F0007C19
:1028AC0007786675F0011280795382F8E582240866
:1028BC00F582BC040390F400DCEC90F4187888D218
:1028CC00F112807953A8FA121BCB446961676E6FC1
:1028DC0073746963206D6F64650D0A00903F271255
:1028EC002F99E57F0404FC7483122FAF902D9C125A
:1028FC002FB6D20D5389F0438901D28C903F11121F
:10290C002F99902DB6122F99200D0A742012251C88
:10291C00902DB28008741012251C902DAE122F9998
:10292C00E57F04B40203E480050303145403F54863
:10293C00754900754A007549007590FCD2EC200D64
:10294C0005122A3B80031229A3C2EC122BB1E549D4
:10295C006548054960147430454912251C7C06797C
:10296C004012252DF709DCF980E1054AE54AB464EB
:10297C0003754A0074C0122FAF7A00AD4AD21ED232
:10298C00561222C5C2560547E547B46408D20C90CE
:10299C00F8007408F0809FD202B2027B03754640A7
:1029AC00200208122D0B122BA38003122D197C046C
:1029BC007AFB80097546407C087AFE0546200203A6
:1029CC006302FFEABB0406F5C0E5C0800E50084464
:0E29DC00C3F5B0E5B08004F5C8E5C86A8A000E
:1029EA003002036300FF55006004A84646F6E5D8A6
:1029FA00540F60024243E590543C643C60024244F6
:102A0A007E0475A0F07819122B94E824F8F8DEF702
:102A1A0075A0F47811122B94EA23FA122CBDDCA5C6
:102A2A000B122D32122B83BB068F30020122022990
:102A3A00A5C202122D19122B837C047AFB7B03E4B4
:102A4A00122BA380067C087AFE79FCEABB0408F5FF
:102A5A00C0E5C0A8C8801B5013F5B0E5B044C37FD9
:102A6A0000122C4ABF0101F442408022F5C8A8C8CE
:102A7A00E5C07F0049122C4AC849122C4AC8BF0136
:102A8A0006F449C8F449C8694241E8694242EA235E
:102A9A00FAEC30E007E92323F9122CBDDCAD0BBBBD
:102AAA0006A375C00075C800E5D8F4540F6002F596
:102ABA00437C0490F01B785AE8F023F8E58224F866
:102ACA00F582DCF4C2EE90F403E8F0122D28122B02
:102ADA00837C04785A90F019E030E00F0582058271
:102AEA00E015821582B50003C38001D3E54533F5AD
:102AFA0045E58224F8F582E823F8DCDCE545C333B2
:102B0A00F54590F411E030E00905820582E06500A0
:102B1A006003434501D2EEE590543C643CF544A27F
:102B2A0002920ED202D2EE122D32E590F4543C6497
:102B3A003C4244122B8390F411E020E70BC2EE12C0
:102B4A002D28E030E7028003434402C202122D1905
:102B5A00122B83C2B2122D28A20E9202783A122D9B
:102B6A00D390F401E030E00A05820582E0B43A022B
:102B7A008003434310122B8322E5905403B40307C6
:102B8A00C2EC7590FC8002059022E254F1B4010077
:102B9A00B3E54572E433F54522E4F540F541F542E3
:102BAA00F544F543F54522E5415542FD902BDD7C80
:102BBA00045403B40313E493A3FE7F58122C98D24F
:102BCA000FE493524152428001A3A3ED0303FDDCBB
:102BDA00E0800802FC01F303CF043F902D747C14BB
:102BEA00E5400303540FB40F0D7E007F58D20F90B7
:102BFA002D7C7C118013BC1004E5418005BC0802C1
:102C0A00E54213FD500D122C56122C98122CADD2FF
:102C1A000F8002A3A3EDDCDE300F05122CADC20F2C
:102C2A00E5436006122C5F122CADE54460070312DF
:102C3A002C83122CADE5456006122C87122CAD228E
:102C4A0075F0083340010FD5F0F93322E493A3FE5F
:102C5A00E493A3FF22FD30E4077E007F53122C98F1
:102C6A00ED7F42F5F0A2F092E1A2F192E0A2F29297
:102C7A00E3A2F392E27E0180087F4480027F507EC5
:102C8A0000135005FD122C98ED0EBE05F422E549FD
:102C9A006006BE000122232324C32E122FAFEF1297
:102CAA002F9E22D20F79C0E4D9FEC9122CBDC9D5F4
:102CBA00E0F622122CEF4004C2068016200613D238
:102CCA0006100C0F754700B40702B20D7581070292
:102CDA00290022C083C08290F800740CF0D082D000
:102CEA008375470022C006C002C001C000C083C06D
:102CFA008212333AD082D083D000D001D002D006DB
:102D0A002275B0C3E4F5C0F5C8D2EE122D32227591
:102D1A00B0FF74FFF5C0F5C8C2EE122D322274124C
:102D2A007900D9FED5E0FB227C0875A0F07802BCB8
:102D3A00040775A0F47802800ABC03028025BC014E
:102D4A000280207402F2200204747080027460F21D
:0E2D5A007445F2122D2818E230E0070808E256
:102D6800181880F508E82408F8DCC622003700396E
:102D78000038004102410239014101390341033958
:102D88000441043902380237013801370338033760
:102D98000438043743313233343536373839303133
:102DA800323334353600804F5000804C4200C0200A
:102DB80030004C4F4F50004F50454E000D0A002038
:102DC8005041535300204641494C00C3122DE57C25
:102DD80008E813122DE5DCFAD3122DE522CA858AFC
:102DE800F020F7FA858AF030F7FAB392B2858AF0C4
:102DF80020F7FA858AF030F7FA858AF020F7FA8505
:102E08008AF030F7FACA22E4936006A31285FA80A2
:102E1800F622E549600B902EE07C04232304FD8014
:102E280019902DBF200D03902DBA122E0F902DC48E
:102E3800122E0F902EC47C057D00E57FB401021C84
:102E48001CC083C082C001C004C0057A00D2219092
:102E5800E8101222C5C22190E811122E0FD005D019
:102E680004D001D082D0830D7907C3E493A3F8E49A
:102E780093A3566024400FC083C082902DCD122E9C
:102E88000FD082D083D374201285FAE493A31285DD
:102E9800FAE493A31285FA8002A3A3D9CE400CC00A
:102EA80083C082902DC7122E0F8004C083C08290E9
:102EB8002DC4122E0FD082D083DC862240043037F6
:102EC8004010303840083039402031304402313326
:102ED8004501323543105131420830374204303809
:102EE800410830394104313043023131440431332F
:102EF800450232354201303742023038410130391B
:102F0800410231304301313144083133450432350F
:102F180042203037421030384120303941103130AA
:102F28004308313144103133450832354280303757
:102F380042403038418030394140313043043131EA
:102F4800442031334510323590F8007430F074065F
:102F5800F0740CF02290F800740DF02290F80074D0
:102F68000CF02275A0F87900F30975A0F87901E44E
:102F780093A36008B45C02748CF380F3222077106A
:102F8800903F69201B03903F7F122F99A21B921C30
:102F980022E493A380CD75A0F87901645C60046491
:102FA8005C8002748CF32275A0F87900F32275A076
:102FB800F87901E493B45C02748CF3A3DCF5227411
:102FC80080122FAFE576122FEA7420122F9E7A0016
:102FD800AD760DBD00047A017D00D2561222C5C21D
:102FE8005622120AE17C10122FB62290F40F7403B5
:102FF800F090F41FF022903F3D122F9922903F53FA
:10300800122F9922C0E07493122FAFD0E0122F9E96
:1030180022903EFB122F9912305E22903EA3122F6F
:103028009922903ECF122F9912305E229033DB12F4
:10303800352DD21690E85F7479F090E85E1232DC94
:1030480012348922903EE5122F99903F11122F9940
:1030580074C0122FAF22903EB9122F9912307012FD
:10306800333A50FBB407F82212333A40FB12407748
:1030780022305708C25720390312360B22E5536015
:1030880002D322307A10AE56BE2E0EC210C27CC2B7
:10309800507C2D1231D4023171201042BE79217C2E
:1030A800221231D4C250D21090E8377401F090E85F
:1030B80038E01240447C107420F0A3DCFC0231712B
:1030C800BE6ED390E838E004B5770280034001E48F
:0E30D800F07C2D1231D4123195C27A0231757E
:1030E6007445A879B855027451B5061390E837E0CF
:1030F600B40102807614F01240447420F0D322BE4C
:103106004718124061C21090E838E0B57603122FD6
:10311600C790E837E0240AFC80BBBE4804D250D3EF
:1031260022BEC804C250D322BE8000503CBE2E0030
:103136004039BE4800500E90410630500390412061
:10314600EE93FE8011BE7B005021BE6100401CEE56
:1031560030500324E0FE90E837E06411600D124021
:1031660044EEF090E837E004F0D322C27AC322E4BA
:10317600F52CF57AC25EC253D322D27C90E838E5AC
:1031860076F0C2507A48121F361231950231759088
:10319600E838E0FF903FF71231FED221EF2401FD1F
:1031A600E43400FA90E83B1222C5E4F090E83B12C2
:1031B60031FEC221903FFC1231FEEF120AE17C1073
:1031C60012320EEF120AF09040001231FE2290E801
:1031D60050E0F875A0EC7445AB79BB55027451F21A
:1031E600D2E708B8C0027800F2C2E708B8C0027891
:1031F60000DCECE8F0D22722202104E4938001E0F1
:10320600600512321C80F122202104E4938001E043
:1032160012321CDCF322C083C0829040B593FA536D
:10322600027F20E70C305013C25074C8121F56801C
:103236000A205007D2507448121F56C004121F3677
:10324600D004D082D083A32290402E122F992290B0
:103256004018122F99903F27122F9922201169208A
:103266001A41203E02801090E853E0B41E0040054B
:1032760012341F800204F0201A2920191330180A6C
:103286001240B3A2E7B3921B80061240C1B3921B51
:10329600201C05301B0D8003201B08303902D25C30
:1032A600122F851232F59257501E90E853E4F0D251
:1032B6007990E85F7479F090E85E30221990F80012
:1032C600740CF0C257C2222290E85DE014F0701E22
:1032D600A3E014F070187404F015827484F090E87A
:1032E6005FE014F0700890F8007408F0D222221201
:1032F600333A4008C20690E856E4F02290338D93A4
:1033060060F214FE3006028004D3D20622BE0B02FF
:10331600800DBE0C028008BE0E028003BE0F139005
:10332600E856E00430E30A2408B4280050DBF080B5
:10333600D8F0C32275A0F47583F4780D791D7582D3
:103346000E7A0112337AB40F2975820E7A0212337D
:103356007A2410B41F1C75821E7A0112337A242037
:10336600B42F0F75821E7A0212337A2430B43F02CC
:10337600C322D322EAF0E25403FEE354032323429A
:10338600060582EAF0EE22000000000000000E00B2
:103396000000080005020000000000000000010017
:1033A60000000900060300000000000000000F00F6
:1033B60000000A00070400000000000000001000E2
:1033C60000000D000C0B00201A03122FC722201A32
:1033D60003122F8522BE0B0BD270D215C26FC238D4
:1033E600023482BE0C0BD271D215C26FC2380234BF
:1033F60082BE0A2290E835E4F01235E7903F951236
:103406002F99122F64D21AC26FC271C27090353CC6
:1034160012352D023482BE0D15C23EA81F123498F5
:10342600403B122F647491122FAF122FD622BE0A80
:10343600004006203E030234DAD23EC23812397FFB
:10344600122F5DE51FB43D09E577B46300500D808A
:0E3456000C500AE577B409005002800122C232
:103464003E1234BF4007B577028007400512342866
:10347400800CF576C270C271C238D26FD215123484
:1034840089122F6422E490E853F0A3F0A3F0751F8F
:103494003BC23E22B83B02C3227E0090E83BE0CE12
:1034A40075F00AA42E500205F0FEA318B83BEF9065
:1034B400E854F0FDA3E5F0FAF0D32290E855E0F5E6
:1034C400F0B40200500E90E854E020F005600514BA
:1034D400C32260FBD322C23890E854E576F09034DE
:1034E400E812352D90E854E0BE0D0DD26FD215F5DB
:1034F400769033DB12352D22BE0E0814B4FF10E58E
:1035040077800CBE0F1904B5770280034001E4F004
:10351400AF76F57674C0122FAF122FCC8F762212AD
:103524002F859033DB12352D22C083C08290E85A58
:10353400D0E0F0A3D0E0F02290E835E0F8BE0B072D
:1035440004B40E0CE48009BE0C2614B4FF02740DFE
:10355400A95F530107B40D05B905E28010B4040254
:103564008008B40C028003B40B03B902D0F080735A
:10357400BE0A58105415C21A9033DB12352D12347A
:1035840089122FC7122F85122F6422903FAB122F5E
:1035940099903FC1122F999035A712352D90E83597
:1035A400E4F022BE0B028003BE0C1290E835E0F476
:1035B400F0903FD76003903FDC122F9922BE0DFCA0
:1035C40090E835E070B012155580ABBE0DBCE82311
:1035D400F8903BE993F9A3E893F582898312352D9A
:1035E40002360B90E835E0F875F014A424B8F5829F
:1035F400E5F0343CF5837480122FAF7C14122FB69F
:1036040012361612361F2290E85AE0C0E0A3E0C03A
:10361400E022903C6DE893122FAF2290E835E0FC55
:10362400903C23230493C0E0EC2393C0E022903F1A
:1036340011122F99903DD0122F9990E835E0F8900F
:103644003C3E7C00E4A39370030C80F8ECB500F4DA
:10365400122F727429122F9E74D3122FAF122F5D62
:1036640012348990397F12352D22903F11122F99EF
:10367400903DDC122F9974C9122FAF12361F903966
:10368400DF12352D22903DE7122F99903E10122F14
:1036940099E5761237DD74C4122FAFE576122FEA5E
:1036A400E576120AF07490122FAF122F5D90E8376E
:1036B400E4F090E836E4F090E838E576F09036C827
:1036C40012352D2290E837E0FFBE0F080FBF110D11
:1036D4007F008009BE0E221FBFFF027F1090E837D3
:1036E400EFF070097490122FAF740D800724C31289
:1036F4002FAF740E90F800F022EF7036BE0B0A1252
:10370400376604B50010E4800DBE0C5E12376614F3
:10371400B4FF03E50014F090E838E0FF1237DD74DD
:10372400C4122FAFEF122FEA7490122FAFEF120AC8
:10373400F022BE0B0B12404404B47E107420800CA3
:10374400BE0C2712404414B41F02747DF0F8122FEB
:1037540064E8122F9EEF24C3122FAF740E90F8006A
:10376400F022A8770890E838E022BE0A13122F64EA
:103774007480122FAF7C14903D30122FB6023A079A
:10378400BE0D1990E837E0601312406190E837E409
:10379400F07490122FAF740D90F800F022903DE772
:1037A400122F99903DFA122F99E5761237DD1210F7
:1037B400371237EA1210371238037490122FAF12EF
:1037C4002F5D90E837E4F090E836E4F090E838E5CF
:0E37D40076F090383112352D22C0E07491123B
:1037E2002FAFD0E0123A4122780E540F14F5F07444
:1037F200C3122FAF12393212395D90E839E5F0F079
:1038020022F8540FB40400400824FDF5F078038038
:103812000CE8C4540F903A7193F5F0780474CA120C
:103822002FAF12393212395D90E83AE5F0F022906A
:10383200E837E0FFBE0F080FBF030D7F008009BE0F
:103842000E381FBFFF027F02BF020990E839E0B4C1
:10385200030050E090E837EFF0122F64904096E4B6
:1038620093600B122FAF741D122F9EA380F1904014
:1038720096EF93122FAF122F5D22BE0B0A12409ABF
:1038820004B50010E4800DBE0C4B12409A14B4FF34
:1038920003E50014A982B9380AC0E01238FFD0E06B
:1038A20090E838F090E838E01237DD90E837E070C1
:1038B2000E90E838E07583EA4400F582E080031256
:1038C200390DC0E01237EAD0E012380390E837E051
:1038D200FF12387022BE0A1C90E837E070031238DB
:1038E200FF122F647480122FAF7C14903D1C122F94
:1038F200B6023A07BE0DDD90E837E0D25412390D18
:10390200FB90E838E0FEC24A0227F090E839E090E6
:10391200391B93B444004006220102034455F89037
:10392200E83AE0903B429354F0482290E835E0F8C0
:10393200903C7CE89390E830F0903C8BE89390E8E0
:1039420031F0903C9AE8230493F9E8239390E8330A
:10395200F0A3E9F02290E832E0F5F090E830E0FCE4
:10396200C0F0A4D0F0F990E830E0FC90E833E0F841
:10397200A3E029F582E438F583122FB622A81FBEF0
:103982000A00500F75A0E8EEF208B83F131818F2BB
:1039920008800DBE0E028003BE0F3218B83A01082D
:1039A200881F7491203E0274D1122FAF12349840B6
:1039B2000A903F127C03122FB68007D2561222C5FC
:1039C200C2567493203E0274D3122FAF22BE0A0253
:1039D2008033BE0DF7123498403E023BD890E83156
:1039E200E0F890E832E0BE0B0704B5000CE4800971
:1039F200BE0C0F14B4FF02E814F074C9122FAF12F8
:103A02003957BE0A10903F95122F99122F649035A4
:103A12003C12352D22BE0D1B90E835E0F8B40002B1
:103A22008002D254903C0793E8230493C0E0E82339
:103A320093C0E022E4A23892E0FC023AD5E5772472
:103A420001FDE43400FA023AE1E55F540FB40205E5
:103A52007C00023AD5B404047C018077B405F17C81
:103A6200028070E55FC45407903A7193FC80640051
:103A7200000103000290E86EE0FD90E86CE0FA536A
:103A8200020F805B90E904E0FC804890E86AE0FD68
:103A920090E868E0FA53020F804590E863E0F4543E
:103AA2001FFD7A00D21E803790E863E0F454600371
:103AB200C4FC801F90E930E0FD7A00D21E80209085
:103AC200E866E0FD7A00D21E801590ED00E0FD7AF6
:103AD20000800C12392D90E832ECF012395722D2C4
:103AE200561222C5C256C21E2290E832E0A2E092CD
:103AF20038023BD21234BF40046002F577023BD257
:103B020090E832E0903B2893F9540FB40209E55F44
:103B1200540FB40202A95F895FC00012067D12072A
:103B220081D000023BD212445590E832E0903B42F1
:103B320093F55FF9895FC000120781D000023BD282
:103B42001222523290E855E090E86CF0A3F090E82F
:0E3B520054E090E86EF0A3F0807690E832E048
:103B600090E904F0806C90E855E090E868F0A3F0EC
:103B700090E854E090E86AF0A3F0805690E854E0B2
:103B8000F4541FFC90E863E054604CF0804490E8EB
:103B900032E0F4540323C4FC90E863E0541F4CF07B
:103BA000803090E854E090E930F0802690E854E0CE
:103BB00090E866540FF0801A90E854E090ED00F021
:103BC000FEC000E412251C740312251CEE12251CF5
:103BD000D00012361612361F122F64903F95122F06
:103BE0009990353C12352D2222366E3632366E369D
:103BF0006E366E37A1368936323632363236323646
:103C000032366E363236323AEB3B463B5C3B023B59
:103C10002B3BE83BE83AF63BA23BAC3B663B7C3BAC
:103C20008E3BB83A363A773A863A4B3A653BE83BB0
:103C3000E83A3F3AB63AC13A8D3A9C3AAA3ACC00B1
:103C4000312D393939000000000000322D3235366F
:103C500000312D313600312D313600312D393939D1
:103C600000322D33300000302D323535008B8C8FF3
:103C70008A87D4D48F919191928A91D40300030AB8
:103C80000A00000000000000070003020002030415
:103C9000000000000000000400053E7200003E6CC1
:103CA0003E263E440000000000000000000000002E
:103CB00000003E7800003E945363616E206D6F6497
:103CC000651D202020202020202020205363616EAD
:103CD0002074696D651D20202020202020202020B8
:103CE000506F776572206F6E207363616E1D2020A8
:103CF000202020204B6579626F6172641D20202096
:103D000020202020202020204D6F7573651D20204D
:103D1000202020202020202020202020435055201B
:103D20006B6579626F6172642F6D6F7573652020AA
:103D3000435055206E616D65732020202020202087
:103D4000202020204D6178696D756D20706F727430
:103D5000731D202020202020457870616E73696FCC
:103D60006E2077696474681D20202020457870617A
:103D70006E73696F6E20756E6974731D202020202C
:103D8000566964656F20626C616E6B2074696D6545
:103D90001D2020204B422072617465206B65797371
:103DA0002F7365631D2020204B422064656C617970
:103DB0001D202020202020202020202053756E2030
:103DC0006B62206C616E67756167651D2020202025
:103DD000C04E65772076616C75652800C043686FBA
:103DE0006F73659E9F20008043686F6F7365209E90
:103DF0009F7F7E20204350551D00C04B421D202038
:103E000020204D531D202020202020202020200075
:103E1000C04E616D65202020202020202020202001
:103E2000202020202000504320202020202020205F
:103E30004D61632020202020202053756E202020FB
:103E40002020202050532F32202020202020536576
:103E5000724D6963736F667453657250436D6F750D
:103E60007365536572204F74686572204E6F2059D8
:103E700065734F66664F6E20536C6F772020204D20
:103E8000656469756D2046617374202020466173F6
:103E9000746573745043315043325043334D616302
:103EA00053756E80526573657420737563636573B3
:103EB0007366756C2020202000C048697420656EF0
:103EC00074657220746F2070726F63656564008022
:0E3ED0005265736574206661696C656420201C
:103EDE002020202020200080436F6E666967757257
:103EEE006174696F6E207265736574200080436F14
:103EFE006E66696775726174696F6E2062616420A7
:103F0E00202000C020202020202020202020202023
:103F1E002020202020202020008020202020202053
:103F2E00202020202020202020202020202000C003
:103F3E0050726F6772616D20636F72727570746507
:103F4E006420202000C0536C617665206C696E6B16
:103F5E002062616420202020202000C053746174F0
:103F6E0075731D206E6F726D616C202020202020D5
:103F7E0000C05374617475731D206E6F206370756D
:103F8E0020706F77657200C0456E746572A573659B
:103F9E006C656374209E9FA56974656D0080536186
:103FAE00766520636F6E66696775726174696F6E90
:103FBE00202000C0456E7465722063686F6963656A
:103FCE009E9F20596573202000CF59657300CF4EF8
:103FDE006F2000805363616E206D6F64652020201A
:103FEE002020202020202020004E616D6500203DE5
:103FFE002000204368616E676520592F4E2F455370
:10400E00433F20004F6E204F6666C0537461747537
:10401E00731D206E6F742073656C65637465640028
:10402E00C05374617475731D20766964656F206F5B
:10403E0066662020200090E838E05403C4F890E82B
:10404E0037E014540F42007583EB7400543F48F56B
:10405E0082E02212098290E838E0120AE15382C00F
:10406E0075A0EB79001216A82278007900D9FED837
:10407E00FC2290E837E4F0FF12408A22904096EF3F
:10408E0093122FAF122F5D2290C2C900BF01077885
:10409E000590E839E022780490E83A5006A87708AF
:1040AE0090E838E022E575C4540F4410F58275830C
:1040BE00E9E022C0E0740925748355D8D36001C3AA
:1040CE00D0E0220201080444B1C0B3B4B5B740B980
:1040DE00B0B8BB413A4243303132333435363738DB
:1040EE0039BF3FC13BC2C3B2E1E2E3E4E5E6E7E834
:1040FE00E9EAEBECEDEEEFF0F1F2F3F4F5F6F7F8AA
:10410E00F9FA3C3E3DB6BA2F616263646566676834
:10411E00696A6B6C6D6E6F70717273747576777889
:10412E00797ABCBEBDAF1B60303132333435363791
:10413E0038392D3D5B5D5C3B272C2E2F2008090D59
:10414E001B7E2921402324255E262A285F2B7B7D7A
:10415E007C3A223C3E3F2008090D2030382F323960
:10416E002F393920436F707972696768742031393D
:10417E0039302D3139393920526F736520456C65D0
:10418E006374726F6E69637320C2A91291DD75F04C
:10419E002C1242781242991242BE20083F1242451A
:1041AE00403AD20ED279A950A7060953016FA7073C
:1041BE00B7FF02800EB7B607E506B4B60280040953
:1041CE0053016F895030011474201285FA744B120A
:1041DE0085FAE5061285DCE5071285DC1291EA12F6
:1041EE008B5AD2A922128B85C2A91291DD75F03C91
:1041FE001242781242991242BE20083212424540B3
:10420E002DD20DD279A959A7060953014FA7070937
:10421E0053014F8959D249300114744D1285FAE574
:10422E00061285DCE5071285DC74201285FA1291E0
:10423E00EA128B5AD2A9221242CE402D7D0812428A
:0E424E00CE4026300903C38001D3E50633F5C8
:10425C0006DDED7D081242CE4011300903C380010A
:10426C00D3E50733F507DDED1242CE2253B0CB7CFC
:10427C0092000000DCFB43B0347C1ADCFEE5F07DE0
:10428C00083312431C0000000000DDF52253B0CBB4
:10429C007C1FDCFE43B0347C0DDCFE20B4028004B9
:1042AC00C208800D7CFF20B406DCFBD2088002C261
:1042BC000822C2087C3F30B406DCFBD2088002C264
:1042CC0008227CFFDC02801D20B4F97C000C30B489
:1042DC00FCC3EC940E500AC3EC94034008C2098052
:1042EC0002D209C322D3227C26DCFE227D10C5F02B
:1042FC00D312431C000000000000003312431CBD0D
:10430C000904C5F08003000000DDF0C312431C2239
:10431C00C0E053B0CB7C0D500280027C1BDCFE4312
:10432C00B0347C13500280027C05DCFED0E0227C91
:10433C00127DFFDDFEDCFA22128B85C2A91291DD03
:10434C0075F02B1242781242991242F375F0627595
:10435C00E0031242F81291EA128B5AD2A9224300BE
:10436C00F830E0055300FB800343000430E10553B3
:10437C0000FE800343000130E2055300FD8003433F
:10438C000002E5002212436A85E0827583FF128BDE
:10439C0085C2A91291DD75F02A1242781242991247
:1043AC0042F38582E08583F01242F8C20C1291EA46
:0443BC00D2A922223E
:1043C00002979232FFFFFFFFFFFFFF758C10D26B49
:1043D000327583F011607583F4116012873D7900A6
:1043E0007583E8E92480F582E07583EAF582E012BE
:1043F00080CA09B904EA90F400786675F000E55FB8
:104400005407117990F410117990F408787775F0C9
:1044100003117990F41A7415F07582187403F02260
:1044200075821274C0F075820FE075821FE075828C
:10443000047470F0758214F022438202741AF0F052
:104440005382F8438200741330F2027407A2F09290
:10445000E0F07407F05382F8438201E8F05382F8E9
:10446000438202748020F1027490F074A020F10263
:1044700074B0F07405F05382F8438201E030E00933
:104480005382F8438203E080ED22C4540F75F0009C
:104490007866B40500401AB4050575F0018012B4C1
:1044A000060775F00578668008B407F375F00178A3
:1044B000997583F0E9C403F58212807922E590545E
:1044C0003C537DC3427D227583F030E3037583F452
:1044D000C4032401F582E030E20D5382F8438203E5
:1044E000E8F0129056C322D3755D0022E8B578003B
:1044F000401B9093E793FE55906004EE427D22EEC0
:10450000557D6009E8784D3107EEF4527D22F9E5DA
:1045100074B11B74EFB144E574B11BE9B144227965
:10452000387B30D255E95403C074F574B1C8D074E7
:104530005002805DE578601DE95403F8B5780050BD
:10454000047412803190E930E08578F0A428C39596
:1045500078F5828007E954032400F5827583EAE048
:104560005407B407051283F68027B4040280224062
:10457000047135801CE0C0E0F16E430104F16E531C
:1045800001FBD0E054F0B450028006E95403F83146
:104590002C090B309803128BC4B93C89C2552212E6
:1045A0008FC51285C8204E49404720020320182B92
:1045B000E5795407B40707E574128107802AB4042B
:1045C0001175F0FF12909150280554E554B4022A59
:1045D000801F4007E5741286378016E57412851B2C
:1045E000E890E885F012855D50070554E554B4A0C5
:1045F0000975540005551553C322D3221285C820CE
:104600004E565002805220020320183EE579C454D1
:1046100007B4041888F009E3F81290A6500A055D63
:10462000E55DB4023A755D00755C00224012B40786
:1046300007E5741286A78020E574128107501922BD
:10464000B40207E57412810780F3E5749093EB934D
:10465000557D60041282A022755D00055E155C2206
:1046600075A0E8A85EE574C2E29085C49345C0B425
:10467000FF4AE574D2E212851B128B85E574C2E213
:104680009085C49345C0B4FF2F12830B20010440D2
:10469000278018742E400274201285FA74781285CF
:1046A000FAE2C0D01285DCD0D0400D055E08D55CA2
:1046B000D8755C00128B5A22128B5A22742D1285E7
:1046C000FA74781285FAE21285DC22E2C31284C6FB
:1046D000306514A2D0B37C09131284C6306508DC9F
:1046E000F7D31284C6C322D3FCE572F442C8E57343
:1046F000F442C0EC22E754036002801AE95403122A
:104700008440400122B710057700715822B4013966
:1047100077037E00715880737583E9E95403F84488
:1047200010F582EEA2E292F0A2E092F1A2E392F200
:0E473000A2E192F3E5F0540FF0E576200205C9
:10473E00E575C4540FB50044D25C22B40E06771052
:10474E00128A6422B40F0477068032B402028010FB
:10475E00B40302800BB40A028006B40B028001225D
:10476E00E95403F8E576200205E575C4540FB5004B
:10477E000B90E8402582F582EEF0D27522E79097F5
:10478E008993B4040E90ED00E0A2E77404500D740A
:10479E00038009B45A0690ED00E0547FF8E9540303
:1047AE0012863717128A642290F41112842950113E
:1047BE007420B1FA746BB1FAE8B1DC90F001128496
:1047CE003690F00112842950117420B1FA7463B13D
:1047DE00FAE8B1DC90F40112843622E020E002C344
:1047EE0022438203E0F8D322E030E2FC438203E866
:1047FE00F0227583F0F830E3037583F4C4032401CB
:10480E00F582E020E004C3E4800B5382F843820378
:10481E00E012905BD3FE22A2E2924AC0E0B11BD01E
:10482E00E0540390854093C002FA128B857C087881
:10483E000091E4E5C8304A02E5C05AC36001D3EEE8
:10484E0013FEDCED91E4E5C8304A02E5C05A600182
:10485E000C91E4E5C8304A02E5C05AC24A6002D261
:10486E004AC391C6E572F442C8E573F442C0128B96
:10487E005AD002ECA2E0EE22C0E0400AE57252C825
:10488E00E57352C0800AE572F442C8E573F442C083
:10489E00D0E07F0180027F04DFFEC0E0E57052C8E9
:1048AE00E57152C07F0EDFFEE570F442C8E571F48B
:1048BE0042C0D265E570F4600855C88009C0E0803A
:1048CE00F1E571F455C07002C265D0E022FE2055AC
:1048DE000430190122A2E2C2E290853C937FFF4090
:1048EE0001CFF57103F573CFF57003F57222F7FD65
:1048FE00DF7F04011040C00179027D00C0E01290FC
:10490E006F128573D0E05004DDF2D9F0D001222071
:10491E005506301903022488BE0400500512903348
:10492E008003129047FFEEA2E2C2E29085C493404C
:10493E000445C8800245C0CFBFFF028002D32212B9
:10494E008B8512850B30651EC31284C6306517A287
:10495E00D0B37C09131284C630650BDCF7D31284F6
:10496E00C6C3128B5A22D3FCE572F442C8E573F427
:10497E0042C0ECD380ECF3FCCF3FC0E07409257449
:10498E008355D8D36001C3D0E02202010804300160
:10499E0011C0E0C4540FB1F1D0E0C0E0540FB1F13A
:1049AE00D0E022B40A00400224072430300107F57B
:1049BE00993099FDC2992290E857E0D5E00274062D
:1049CE00F0B406247938E7B4200280045407600F4F
:1049DE00B24020400A77005301F77700430108E503
:1049EE002803F52809B940DE22C8129060C89097B6
:1049FE006F93FAC3D1507C08E813D150DCFBD3D1AE
:104A0E005022CA858AF020F7FA858AF030F7FA40EC
:104A1E000452C88004F442C8F48024C8129065C8B9
:104A2E00C3D17D7C08E813D17DDCFBD3D17D22CAB6
:104A3E00858AF020F7FA858AF030F7FAB392B285BC
:104A4E008AF020F7FA858AF030F7FA858AF020F797
:104A5E00FA858AF030F7FACA22C8129060C8909789
:104A6E006F93FAC3D1C47C09E8A2D0B313D1C4DCCE
:104A7E00FBD3D1C4C322CA858AF020F5FA858AF009
:104A8E0030F5FA4006F442C8F4800252C8858AF026
:104A9E0020F5FA858AF030F5FA858AF020F5FA8548
:0E4AAE008AF030F5FACA22AC7420020CE575CD
:104ABC0054C0701FE575C45403FC74382CF82404DE
:104ACC00F9E6B42001225407700BE7B420012254FC
:104ADC00077002D322C322C320020DE57554C070A7
:104AEC000EE575C454038002E576B50402D322C3E7
:104AFC00227C0075A0E87880EC20021F12872340EE
:104B0C001890E930E0F5F0ECB578005003A4800B78
:104B1C00E578A42CC395788002E576F2080CBC04E9
:104B2C00D722E9540390854093FAE9A2E2E5C850F4
:104B3C0002E5C0FE5A7044EE035A603F5012E5C8BD
:104B4C00FE5A7007EE035A70028030E5C05A702B83
:104B5C00E954079165304A0F20D0045004800A5064
:104B6C00087433C24A80027422B93C00500512907A
:104B7C0038800312904C304A02800302885CE7B400
:104B8C00200CE920E22EBEE000403402889EE93081
:104B9C00E2F91287F5B4EEF3BEEC0302889EBEFF79
:104BAC000302889EAC060288B8540390E87C2582E8
:104BBC00F582E0221287F5B4F305128A734051771F
:104BCC0019E920E24B540390E840FC2582F582E081
:104BDC00B4ED20EE7583E98C82438210F0128723AA
:104BEC00502EE07583E98C82438210F0D25C0289EE
:104BFC0000805FB4F01AEE701AECB57800857682FE
:104C0C0040028C827583EAE05403232323242AF781
:104C1C000289F7128A525407D2F0B40400501FEEE6
:104C2C00A2E792F030020D30E70AA2E45403B392EB
:104C3C00E4F0800AE054F05306034EC2E7F012870A
:104C4C00235071301805A2F0B39207E0F579D25DCC
:104C5C0080629093657C8BB93C0040059093897C75
:104C6C00ABA3A3ECB58250B4AB077CFEE954078030
:104C7C0012BEFE19E954037CFAB5740790E885EC72
:104C8C00F0E57412851BEC12855D0289F7128A52CD
:104C9C00B45506EE128399801775A0E8E9540324E5
:104CAC0040F8E2F87451B8FE005014B8FB00400F05
:104CBC00741977190289F7E493B506A5A3E493F761
:104CCC00E95407A2E2C2E290E840500390E87C2548
:104CDC0082F582EEF0E9540730E21DC2E2B5742E83
:104CEC00C0E0C3E559955A540F20020F204D0C75A6
:104CFC00F0038475F003800A0289D675F00484757C
:104D0C00F004A4255A544FF55A755C00D0E0BEF25D
:104D1C0024E95403B57800400C128A5254F07012F6
:104D2C00776A0289F7304D02776A5301FB777A4331
:104D3C0001040289F7D2E2BEE924750504F5007C72
:104D4C001EE812851BE505240F83C00412855DD077
:104D5C00045002DCECD505E780513C0390FA9093AB
:104D6C00EB540393BEF404427D8040BEF50B201837
:104D7C00F82019F5F4527D8032BEF6028003BEFF96
:104D8C00E8C0E0128B13D0E080E4BEFF1E7583E90F
:104D9C00E95403F582438210E4F0128A5254F04431
:104DAC0002F0E95403FC128723925CE75407605528
:104DBC008B0006E6FEE7B40F0050079092D7936E77
:104DCC007043E9A2E2E5C85002E5C0035A7003162D
:104DDC008033E95403C074F5741285C8D07440252F
:104DEC00E9540712851BE79092E793FCE95407B549
:104DFC00740590E885ECF0EC12855D500316800587
:104E0C001776005164227583E8E954032480F582F7
:104E1C00E07583EAF582E022E924CB83522822FE56
:0E4E2C00FDFBF7EFDFBF7FBEC803028AFCBEAE
:104E3A006408128B03B4C8788078BE5008128B03BA
:104E4A00B4646D8049BE14028068BE2808128B03C0
:104E5A00B4145D805DBE3C58128B03B42852128A8A
:104E6A00FAE95407F5007505087C1EE812851BE56A
:104E7A0005241183C00412855DD0045002DCECD5F0
:104E8A0005E77700D322030B0B0B231F32FAC3C0AB
:104E9A00D0128A52D0D0540F50024410FEE9540363
:104EAA00B57800400BCEF0CEFC12872350028E79E3
:104EBA007E00128B08EEF0C322128B08E02290E8E3
:104ECA0078E954032582F58222C006D3128AD97E54
:104EDA0000128AFCD006222018352019321285C801
:104EEA00204E2C402AE579B4440975F0FF78B612B1
:104EFA00909122B4550FE574784C128637E5747890
:104F0A00CC12863722B47707E57478B31281072268
:104F1A0020022530AF24C0E0203B12E55F644460E4
:104F2A0015E55F6455600FC289D2A8D2B2203A064D
:104F3A00C28BD2AAD2B3D0E0D2A92220023530AF96
:104F4A003430A816202FFD203B10C2A87CFF20B2C7
:104F5A0004DCFBD266C2B275250830AA162037FDDA
:104F6A00203A10C2AA7CFF20B304DCFBD267C2B38A
:104F7A00752608C2A97C32DCFE22200236205E3366
:104F8A00205930205A2D20582A203D27205C2420E1
:104F9A005D21203C1E205B1BC3E5592410955A5401
:104FAA000FB40900500DE599C298201207B43F04C6
:104FBA0085769922F5993099FDC29910124C205E96
:104FCA0048B40005D212C22022B40105D212D2205E
:104FDA0022F890E852E0C8B40D1518E577B500003C
:104FEA00400A8876C270C238D26FD215E4F0222401
:104FFA00D0B40A005013C8C0F075F00AA4D0F0303B
:10500A00D2028005285001E4F02220200AA850F696
:10501A000853006F885022A859F60853004F885940
:10502A00D24922855600755300E579540FFE3002A5
:10503A0002800C3018097E03B4030050027E027508
:10504A00A0E87920BE0402801FB81A028003B89A29
:10505A0017EE142323FE9093AB755300EE9360076B
:10506A00F3090E055380F522E86007A2E792F002E1
:10507A008D00BE0303028D484011E557A2E792F066
:10508A00C2E7B4190040EEF8028D87E557B405006F
:10509A0050E374E0F309755301E5571423255714B7
:1050AA00F89093CBBE01039093BFE8936007055332
:1050BA00F3A30980F522BE0133E8547FB40F0C3004
:1050CA00F002803A9093D7780080DFB1AF6009A2EE
:1050DA00F092E7F3755301229093EF74E0F309E835
:1050EA00547F93A2F092E7F375530222BE0247E877
:1050FA00547FB41F03301806B40F0E30F0047553F2
:10510A0000229093DE780080A1B1AF600F75530141
:10511A0030F00674F00553F309E8F32290946F75A2
:10512A00530274E0F30930F00974F00553F309539C
:10513A00007FE893F322BE0304B1AF80D0BE04041B
:10514A00B1D78003BE051DE5567014B81905BE0413
:10515A00AD8003BE05A890975AE8C2E793A119B19A
:10516A00AFA1192222EE149094EFC0F075F080A43A
:10517A0024EFF582E5F0D0F03494F583E8C2E793A2
:10518A00B4FF06D0E0D0E0A1486001F822B81A03C3
:10519A00D38004B89A0AC3128FEE92E2F0D25C224C
:0E51AA00B87C17128FEED25CB2E2F0D2F07831
:1051B800FC30E207C2F0787C75530122B8FC06D0B7
:1051C800E0D0E0A148B87B07128FEEB2E18008B8C2
:1051D8000E08128FEEB2E0D25CF022D27375A0E80E
:1051E8007928E579C4540720193030180520072795
:1051F8008028B40706F17E755C0322B40406D165E5
:10520800755C02224006D18F755C0522B40206F156
:105218003A755C03226003D1ED22D1F12290E82D8A
:10522800E0F5F0A3E0A2F492E6D2E790E829F09046
:10523800E82FE0A2F592E7F404A2E792E6A2F0B321
:1052480092E790E828F02290E82DE0F875F080F4D5
:10525800A2E092F2A2E192F0A2E292F1E5F090E8E7
:1052680028F088F0A2F490E82EE090E829D1C3A2B3
:10527800F590E82FE090E82AD1C322401420E704F3
:105288007800801B04F853007F7002787F747F8059
:105298000EB48000400478008005D2E7F87480F0EE
:1052A800A3A3E8F022740380027404FCF55C90E880
:1052B8002D75A0E87828E0F208A3DCFA22A85A9015
:1052C800E82D7C0374201285FA74751285FAE612AB
:1052D80085DCF008A353004FDCF4200209203906CE
:1052E800204D03E48002E608F01285DC53004F8865
:1052F8005A2290E82DE075F040A2E092F5A2E192E2
:10530800F4A2E492F1A2E592F390E82EE0A2E692EC
:10531800F0543F90E829F090E82FE0A2F392E7F4E8
:1053280004A2E692F2A2E792F3543F90E82AF090A2
:10533800E828E5F0F02290E82DE075F090A2E092E0
:10534800F2A2E292F1A2E192F0A2E4B392F4A2E511
:10535800B392F390E82EE07002D2F430E702F4043E
:1053680090E829F090E82FE07002D2F330E702F4D9
:105378000490E82AF090E828E5F0F02222E5795434
:1053880007B40404747F80044017743068A2E7C22D
:10539800E7700EE574908FEA934004F452C02242FD
:1053A800C02208022080E576200205E575C4540F66
:1053B8004410F5827583E9E022751E748076751EA7
:1053C800738071751E53806C751E6D8067751E2AFB
:1053D8008062751E2B805D751E798058751E7A80D7
:1053E80053751E6B804E751E4B8049751E63804435
:1053F800751E43803F751E78803A751E5880357536
:105408001E708030751E50802B751E758026751E87
:10541800718021751E51801C751E628017751E4291
:105428008012751E72800D751E778008751E6D803E
:1054380003751E6E300111C0E074201285FAE51E56
:105448001285FAD0E01285DC22C20DD20EB87F0593
:1054580075F07F8005C5F0C8C5F012923E22D20DC6
:10546800C20E30010CC8129079C8C5F0129079C5E7
:10547800F012923E22C20843C83E7C0FDC02804DE7
:105488007DFFE5C8553C6004DDF880F07C000C0029
:1054980000E5C8553C60F7C3EC9467500A20082D16
:1054A8001292CED20880D07C000CE5C8553C70F929
:1054B800C3EC9409500280157D081291B2400E3059
:1054C8000903C38001D3E833F8DDEFC322D322E513
:1054D8003F52C8E53D52C07C68DCFEE53C42C0E571
:1054E8003E42C82200E8B42A06D20BD20C802DC254
:1054F8000BB42C09300E1FC20ED20F801BB43C090E
:10550800300D13C20DD20F800FB42E0A8EF08FE02B
:10551800C20ED20F8002C20F7C5FDCFE227D10C556
:0E552800F0D312918900000000000000331241
:105536009189BD0904C5F08003000000DDF0C312A7
:10554600918922C0E0E53F52C8E53D52C07C0B5030
:105556000280027C19DCFEE53C42C0E53E42C87C86
:1055660013500280027C06DCFED0E0227CFFDC02C7
:105576008023E5C8553C70F67C000CE5C8553C60B8
:10558600F9C3EC9408500AC3EC94044008C209809D
:1055960002D209C322D322853C1E853D1D853E1CB1
:1055A600853F1B22851E3C851D3D851C3E851B3F78
:1055B600227C26DCFE80151291B2C2087CFFE5C86B
:1055C600553C6006DCF8D2088002C208221291B26D
:1055D60040257D081291B2300903C38001D3EE3312
:1055E600FEDDF17D081291B2300903C38001D3EFCD
:1055F60033FFDDF11291B222888285F083128B850A
:105606001291DD1292A51290BD402A129282500B81
:105616001291178582E08583F080EB12912C200B86
:105626000E300F118582E08583F012916580061297
:1056360091F71292131291EA128B5A22200D0280D0
:1056460003200E16E854F0B400028011B4200520A1
:105656000D0B8006B43006200E03C38001D322C092
:1056660082C083E5749092C693F53C64FFF53DE5F0
:10567600749092CA93F53E64FFF53FD083D08222A0
:10568600040110400C0330C07C047DC8DDFEDCFA4A
:1056960022000A01000000000000010301000000D2
:1056A6000000AAFA00000000000000AAFA000000AC
:1056B600000083ABFA0000000000FA0000000000C2
:1056C6000000FA0000000000000000FA00000000E0
:1056D600000001FA00000000000002FA00000000CD
:1056E600000003FA000000000000EE0000000000C9
:1056F6000000FE00000000000000BFB0FA0000003D
:105706000000000008FA0000000003FA0000000094
:105716000000FC0000000000000000EF0000000098
:1057260000FF02F213ED21F321F419F021F519F629
:1057360019F719F819F919FA19FB19FC19FD19EED7
:1057460049D251EF5BFF0BF619F519F419F321F263
:105756002AE821E719E619EA19E900EC19F019EE29
:1057660019EB64E4713ABA000058F0580014F014CA
:10577600000000000077F77F002A0000360000AA2C
:105786000000B60000120000590000F01200F059A7
:1057960000E11D45E19DC500E11477E1F014F077C5
:1057A60000040810200102408000000000000000F4
:1057B60000000000000037000000000000000000AC
:1057C6000000000000005D00000000000000000076
:1057D60000000000000000000000000000000000C3
:1057E60000000000000000000000000000000000B3
:1057F600000000001D00385B5C5253474F4951487A
:10580600504B4D00350000001C0000000000000059
:105816000000000000000000000000000000000082
:10582600000000000000004600000000000000002C
:105836000000000000007C000000000000000000E6
:105846000000000000002F00000000000000000023
:105856000000000000000000000000000000000042
:105866000000000000000000000000000000000032
:10587600000000001400111F2770716C697D7A7595
:10588600726B74004A0000005A000000000000001D
:105896000000000000000000000000000000000002
:0E58A600000000000000007E00003B3C3D3E84
:1058B4003F404142434457580046FF524F50514BDA
:1058C4004C4D474849FFFF5600FFFF2BFFFFFFFFEA
:1058D400FFFFFFFFFFFFFFFFFF01290B020304058A
:1058E400060708090A0C0D1A1B2B272833343539EF
:1058F4000E0F1C2A361D00380000000000000000B6
:105904000000000000FF00374A4E00531E302E20D6
:1059140012212223172425263231181910131F149B
:10592400162F112D152C453A5400FF000506040CC2
:10593400030B830A01097807007EFF7069727A6B92
:1059440073746C757DFF60610062625DFFFFFFFF31
:10595400FFFFFFFFFFFFFFFFFF760E45161E262504
:105964002E363D3E464E55545B5D4C5241494A29C4
:10597400660D5A12591400110000000000000000C6
:105984000000000000FF007C7B7900711C322123A1
:10599400242B3433433B424B3A31444D152D1B2CBD
:1059A4003C2A1D22351A77588400FF00070F171F61
:1059B400272F373F474F565E575F627069727A6B85
:1059C40073746C757DFF80138D818153FFFFFFFF1E
:1059D400FFFFFFFFFFFF80FF82080E45161E2625EE
:1059E4002E363D3E464E55545B5C4C5241494A2945
:1059F400660D5A1259115819398B8C67646E656F8C
:105A04006D6360616AFF777E847C79711C32212327
:105A1400242B3433433B424B3A31444D152D1B2C3C
:105A24003C2A1D22351A7614FFFFFF007A7863762C
:105A340060616264656D676F696B7152535455564A
:105A44005758595B5C39370A7F7F7F2AFFFFFFFF76
:105A5400FFFFFFFFFFFFFFFFFF35321D1213141579
:105A640017161A1C191B18211E2A29272B2F2C3113
:105A7400333024383836363A3A3737727573777498
:105A8400793E3D3B3C514B434E454C41000B080293
:105A94000E030504222628252E2D1F230C0F011189
:105AA40020090D0710064739FFFF39000506080ACB
:105AB4000C0E10111207090B1617155E7071725B2C
:105AC4005C5D444546FF787C30303058FFFFFFFF73
:105AD400FFFFFFFFFFFFFFFF7F1D2A271E1F20215F
:105AE4002223242526282940415856576B6C6D796A
:105AF4002B3559636E4C43130D787A2C42344A602B
:105B04007B141B181CFF2E2F477D5A324D68664F9D
:105B1400385051523D5354556A693E3F36394E3AD6
:105B24003C6737653B646277FFFFFFFBFEEFBF51C5
:105B3400762D02040103191A313348495F61300F8D
:105B44007374757F6F007F04FF005AFE000075B008
:105B5400FF75810775E80475D8DF7590FCE4787FDC
:105B6400F6D8FDE590F454C02440F57F60FEE0745F
:105B7400FFF575755060755160755940755A4075DB
:105B84007B00757C0090E8577406F0D202129C5F8B
:105B9400B4E6FA129C5FFC90ED00129C5FF0A3DC6B
:105BA400F9E57FC4FE90E9107C04129C5F602AFF33
:105BB400540CD2F0B50602C2F0129C5F20F0EBF058
:105BC400A3DCE77C04EFC4540FB4000590E9208003
:105BD400D9B401D690EA0080D11280111280FD530D
:105BE40089F0438901D28CD2A9D2AF437DC3306BF3
:105BF40003129BFB306D09E55C7005128FC4C26D06
:105C04001286F54003029BB1E57BB57C02802675C4
:105C1400A0E8A87CE2F9E57412851BE912855D50C1
:0E5C2400090554E554B4A008800608B8100223
:105C32007800887C029B2875A0F47819E220E003A2
:105C42000299FD781B30E503029903E27003029981
:105C520044B4FF28307BE91299A5B481E3129991EB
:105C620010E612A95077000953016FF70953016F2B
:105C720089500299F8F57EC2640299D2307BC1F54F
:105C8200F054FCB428281299BBB481B4129991F94A
:105C920075A0E8A87B30F10574E012998930F0050F
:105CA20074F0129989E9129989887B0299F81299FC
:105CB200A5B4814BA950A7F00953016F89500299ED
:105CC200F87C04A959781BE2FE307B33C3E55924E2
:105CD20010955A540FB40C00748340027484129CC1
:105CE20048B4831BEE80097819E230E0FC781BE2AD
:105CF2001285DCF70953014FDCED89590299F8024C
:105D020099FD129991A2E792235000F57E537E7F6E
:105D1200C264547FB401028013B43002800EB40313
:105D2200028009F85300F0B84015D2767819E230B3
:105D3200E0FC30E503029903781BE2F57AD2642095
:105D4200234ED27C0299FDF208B810027800227824
:105D520019E230E0FC20E504781BE222D0E0D0E03A
:105D6200029903C3E55024109551540FB40E0074E8
:105D72008140027482129C4822E550B551F5E553E8
:105D820070F1C3E57B2410957C540FB40C0080DFC6
:105D9200307B2875A0E8A87B74EF129989E57E1202
:105DA200998930640F307607C27674EF129989E5CB
:105DB2007A129989887B7480129C48107C03029B1A
:105DC20028E57EB4012FC207E57AFE54F0B5061429
:105DD200E57F6E54C0700DEEF5755430C4F576D281
:105DE2006F029B23C27B7575FF7576FF74AA42C052
:105DF200C2EC029B28B4160C7440B57FE774801283
:105E02009C4880E0B40309E57A90ED00F0029B28FB
:105E1200B40405D24D029B28B40505C24D029B284D
:105E2200B43019E57AC454C0B57F0EE57A540390B4
:105E320093EB93457DC57DD26D029B20F95301F012
:105E4200B94026F9C4657F54C0701CE95403F93087
:105E52007B06B57403857A797583EA4400F582E599
:105E62007AF01280CA807A807DB40924207B028075
:105E72006D128FEEF8129BF0540FC44200C074856D
:105E820076741285C8D074B3E892E7129C488056A3
:105E9200B40C07307B02D2EC8044B40208C2EC742A
:105EA200AA42C08039B43119307B14E579540FB459
:105EB2000400500BE574D2E212851BE412855D806A
:105EC2001DB4321A307B15E57954E0700F755C020F
:105ED200755E2890E82874AAF0A3E4F08000307B75
:105EE200057480129C48306F24E55C6015207209AD
:105EF200D27290E83FE4F0801490E83FE0B40200F0
:105F0200400BC27285595A755C00129C25E553708C
:105F120024E550B551028027A851E6F556085300F2
:105F22006F700686570853006F8851128C6DE553C7
:105F3200600D75552075A0E8A855E2F81281DF3092
:105F42007302800CE559B55A028005128F05D2738F
:105F5200E55C7011307318128E23C273E55C600F1A
:105F6200755E28C27375A0E8A95EE3F812823C123E
:105F7200815F105D14105C06107521029832128F39
:105F8200EE4490129C48029832129BF0F85300079C
:105F92000354384844C0129C480298327583E8E59D
:0E5FA200744440F582E0547F129C480298320D
:105FB0007583EAE5764400F582E022C26B1286051D
:105FC000307B1B1285C8B3921B201C05301B0F8031
:105FD00003201B0AA21B921C74A092E0914890E837
:105FE0003FE004F022128B21C26F857674129BF081
:105FF000F57912873DE57444FCF590D27BD2EC1222
:1060000085C8B3921B921C22C0E075A0F47819E2F7
:1060100030E2FCD0E0781BF23001031285FA2275E1
:0C602000A0F47819E230E0FC781BE222CA
:02602C001DDC79
:02602E00580216
:00000001FF
